:100000000C9434000C9451000C9451000C94510049
:100010000C9451000C9451000C9451000C94E50088
:100020000C9451000C9451000C9451000C94B400A9
:100030000C9451000C9451000C9483000C945100CA
:100040000C9451000C9451000C9451000C945100EC
:100050000C9451000C9451000C9451000C945100DC
:100060000C9451000C94510011241FBECFEFD8E026
:10007000DEBFCDBF11E0A0E0B1E0E6E8F5E002C0F0
:1000800005900D92A031B107D9F711E0A0E1B1E0E0
:1000900001C01D92A531B107E1F70E9433010C9414
:1000A000C1020C9400008230910561F0833091050B
:1000B00099F00197C9F416BC80916E00826080931C
:1000C0006E0016C0109285001092840080916F001F
:1000D000826080936F000CC01092B200809170001B
:1000E00082608093700004C081E090E00E94C102B1
:1000F00078949FB7F894809112019FBF8823C9F329
:100100001092120108951F920F920FB60F921124B0
:100110002F933F938F939F938091100190911101A2
:10012000019690931101809310018091120181300A
:1001300091F0209110013091110180911301909163
:1001400014012817390738F081E0809312011092CA
:100150001101109210019F918F913F912F910F905B
:100160000FBE0F901F9018951F920F920FB60F920F
:1001700011242F933F938F939F938091100190911F
:100180001101019690931101809310018091120149
:10019000813091F020911001309111018091130173
:1001A000909114012817390738F081E080931201EB
:1001B00010921101109210019F918F913F912F91F8
:1001C0000F900FBE0F901F9018951F920F920FB6B1
:1001D0000F9211242F933F938F939F93809110013F
:1001E00090911101019690931101809310018091DB
:1001F0001201813091F02091100130911101809114
:100200001301909114012817390738F081E0809389
:10021000120110921101109210019F918F913F9144
:100220002F910F900FBE0F901F901895FC01219AEF
:1002300085E290E09387828785B5836085BD21E064
:1002400030E03587248785E090E090931401809317
:10025000130184B5826084BD89EF87BD3787268707
:1002600080E090E00895CF92DF92EF92FF9280E0DD
:1002700091E00E941601C12CD12C760160E070E063
:10028000CB01609300017093010180930201909370
:10029000030180910E0190910F010E945300E091A3
:1002A0000A01F0910B018081826080838FEFC81A70
:1002B000D80AE80AF80AC701B6010E94D0012FE661
:1002C00032E143E05BE30E945E0220E030E0A901FE
:1002D0000E946C01D6CF5058BB27AA270ED0B4C0BD
:1002E000A5D030F0AAD020F031F49F3F11F41EF4D5
:1002F0009AC00EF4E095E7FB90C0E92FB6D080F3EA
:10030000BA17620773078407950718F071F49EF512
:10031000CEC00EF4E0950B2EBA2FA02D0B01B90123
:1003200090010C01CA01A0011124FF27591B99F06B
:10033000593F50F4503E68F11A16F040A22F232F77
:10034000342F4427585FF3CF469537952795A795C7
:10035000F0405395C9F77EF41F16BA0B620B730B6E
:10036000840BBAF09150A1F0FF0FBB1F661F771FDF
:10037000881FC2F70EC0BA0F621F731F841F48F494
:10038000879577956795B795F7959E3F08F0B3CF1A
:100390009395880F08F09927EE0F97958795089504
:1003A000E89409C097FB3EF490958095709561950F
:1003B0007F4F8F4F9F4F9923A9F0F92F96E9BB27C5
:1003C0009395F695879577956795B795F111F8CF41
:1003D000FAF4BB0F11F460FF1BC06F5F7F4F8F4FAC
:1003E0009F4F16C0882311F096E911C0772321F0A2
:1003F0009EE8872F762F05C0662371F096E8862F3A
:1004000070E060E02AF09A95660F771F881FDAF790
:10041000880F9695879597F9089597F99F6780E8D3
:1004200070E060E008959FEF80EC089500240A9446
:100430001616170618060906089500240A941216BF
:100440001306140605060895092E0394000C11F4F2
:10045000882352F0BB0F40F4BF2B11F460FF04C09F
:100460006F5F7F4F8F4F9F4F089557FD9058440FF8
:10047000551F59F05F3F71F04795880F97FB991F03
:1004800061F09F3F79F087950895121613061406C0
:10049000551FF2CF4695F1DF08C01616170618064D
:1004A000991FF1CF86957105610508940895E89428
:1004B000BB2766277727CB0197F908950BD0C4CFC8
:1004C000B5DF28F0BADF18F0952309F0A6CFABCF3F
:1004D0001124EECFCADFA0F3959FD1F3950F50E022
:1004E000551F629FF001729FBB27F00DB11D639FE6
:1004F000AA27F00DB11DAA1F649F6627B00DA11D8C
:10050000661F829F2227B00DA11D621F739FB00D31
:10051000A11D621F839FA00D611D221F749F3327A1
:10052000A00D611D231F849F600D211D822F762F3A
:100530006A2F11249F5750408AF0E1F088234AF037
:10054000EE0FFF1FBB1F661F771F881F9150504083
:10055000A9F79E3F510570F060CFAACF5F3FECF343
:10056000983EDCF3869577956795B795F795E7956F
:100570009F5FC1F7FE2B880F911D9695879597F980
:060580000895F894FFCF7E
:100586000000000000000AD7233C00000000000025
:00000001FF
